:100000007E07040000000000000000000000000067
:1000100000000000000000000000000000000000E0
:1000200000000000000000000000000000000000D0
:10003000000000004C0A000000000000000000006A
:1000400000000000000000000000000000000000B0
:1000500000000000000000000000000000000000A0
:100060000000000000000000000000000000000090
:100070000000000000000000680A0000000000000E
:100080000000000000000000000000000000000070
:100090000000000000000000000000000000000060
:1000A0000000000000000000000000000000000050
:1000B0000000000000000000000000000000000040
:100EFC004F812000F07F210020A0B70010002000BF
:100F0C0034A0B700400020004420B700840A02003F
:100F1C00000000008E0A0200000000008A1F78000A
:100F2C008B1F78005DFF0700A801200027E7260033
:100F3C000E20ED00FEFF3A001020ED00FCFF3A0001
:100F4C000CFF07004A002800F5FE07001620EF00F2
:100F5C001420EF00D4FF07007A0C280090FF070044
:100F6C002AC0B30074FF07007A0728008CFF070023
:100F7C002813200047D622000E20ED00FEFF3A0079
:100F8C001020ED00FCFF3A00000000000000000003
:100F9C001AC0B30068FF07007A07280080FF07001B
:100FAC0010802000104578008EFD07002AC0B30089
:100FBC0061FF07006A06280079FF070098092000E6
:100FCC00176B29000E20ED00FEFF3A001020ED00FB
:100FDC00FCFF3A000000000000000000CDA2A800B9
:100FEC002AC0B30054FF07008A1228006CFF0700C8
:100FFC0010802000104578007AFD07009809200029
:10100C00176B29000E20ED00FEFF3A001020ED00BA
:10101C00FCFF3A000000000000000000CDE2A80038
:10102C002AC0B30044FF0700AA1328005CFF070086
:10103C0010802000104578006AFD070098092000F8
:10104C00176B29000E20ED00FEFF3A001020ED007A
:10105C00FCFF3A0000000000000000002AC0B300B2
:10106C0035FF07008A0B28004DFF07001080200079
:10107C00104578005BFD070098092000176B2900CC
:10108C000E20ED00FEFF3A001020ED00FCFF3A00B0
:10109C0000000000000000002AC0B30026FF07007B
:1010AC001A0F28003EFF0700108020001045780022
:1010BC004CFD0700C80C2000873927000E20ED00DE
:1010CC00FEFF3A001020ED00FCFF3A002AC0B300EE
:1010DC0019FF07004A0E280031FF0700108020007E
:1010EC00104578003FFD070000802000104078007C
:1010FC000040AF0001003700FBFF37001AC0B300FF
:10110C000DFF07006A0D280025FF07001080200046
:10111C001045780033FD07002AC0B30006FF070016
:10112C008A0828001EFF0700108020001045780058
:10113C002CFD07000020EF0030408800308020009C
:10114C00104078000000AF00050037003080200010
:10115C00104078000040AF0001003700020037005B
:10116C00CDA2A80001003700CDA2A900308020003C
:10117C00104078000020AF000500370030802000C0
:10118C00104078000040AF0001003700020037002B
:10119C00CDE2A80001003700CDE2A900308020008C
:1011AC00104078000060AE00010037000F003700DF
:1011BC002AC0B300E0FE0700008020001040780039
:1011CC000060AF00030037008A082800F4FE070017
:1011DC00020037004A112800F1FE070010802000A1
:1011EC0010457800FFFC0700D4FF37001AC0B3008D
:1011FC00D1FE07008A092800E9FE07002A4080007A
:10120C0002FD07002AC0B300CBFE07003FFD07001C
:10121C001AC0B300E9FC07009A102800E0FE070092
:10122C001080200010457800EEFC070000802000A4
:10123C00104078000040AE00010037000500370078
:10124C00572328000E20ED00FEFF3A00000000009E
:10125C00EAFF37001AC0B300B7FE07005A05280092
:10126C00CFFE07001080200010457800DDFC070041
:10127C0000802000104078000040AE0001003700D4
:10128C00FBFF37002AC0B300ABFE07001420EF00B1
:10129C0006FD0700C200DE00400620000008B80072
:1012AC00F20F2000110009000280D80080017800A4
:1012BC003081200003487800420620000380FB00A8
:1012CC000000510000057800D0FC07000FFD07005E
:1012DC001AC0B300B9FC07009A102800B0FE070032
:1012EC001080200010457800BEFC07005723280012
:1012FC000E20ED00FEFF3A000000000000802000F0
:10130C00104078000040AE000100370001003700AB
:10131C00DCFF37001AC0B30087FE07004A04280020
:10132C009FFE07001080200010457800ADFC0700E0
:10133C0000802000104078000040AE000100370013
:10134C00FBFF37002AC0B3007BFE0700AA1428005D
:10135C0093FE07001080200010457800A1FC0700C8
:10136C00CD82A900C80C2000873927000E20ED0083
:10137C00FEFF3A001020ED00FCFF3A002AC0B3003B
:10138C006DFE07001A13280085FE07001080200050
:10139C001045780093FC0700CD82A800CD62A9000F
:1013AC00C80C2000873927000E20ED00FEFF3A0004
:1013BC001020ED00FCFF3A002AC0B3005EFE0700CF
:1013CC002A14280076FE07001080200010457800B3
:1013DC0084FC0700CD42A900CD62A800C80C2000F7
:1013EC00873927000E20ED00FEFF3A001020ED009B
:1013FC00FCFF3A00CD42A8002AC0B3004EFE070005
:10140C009A10280066FE0700108020001045780016
:10141C0074FC070000802000104078000040AF00F2
:10142C0001003700FBFF37000080200010407800DF
:10143C000040AE000100370001003700C1FF37004B
:10144C001AC0B3003CFE0700EA0F280054FE070048
:10145C00108020001045780062FC07002AC0B30001
:10146C0035FE07008A0A28004DFE07000080200088
:10147C00104078000040AF0001003700FBFF370040
:0C148C00CF0578004F057800FFFF370007
:100CA8000028220042A7B7004427EF00C0FF2F000A
:100CB8002CA3B700F0492000C0A2B700902F200055
:100CC800C8A2B700100C2000D0A2B70042C7A900E4
:100CD8000060200080A6B70042C7A800D522A9005E
:100CE800D522AE00D502A900D522AF00D502A800B2
:100CF800409C200002A1B7000001280004A1B70011
:100D08009460A8008680A9009680A8008220A80088
:100D1800CC42A900CD42A800CD42AE00CD62A900C8
:100D2800CD42AF00CD62A800CD62AE00CD82A90051
:0C0D3800CD62AF00CD82A80000000600D4
:100B80008A1F780068062000B79C2B000E20ED001D
:100B9000FEFF3A001020ED00FCFF3A0000000000CC
:100BA000C122A900C102A900D042A900D022A900F7
:100BB000D482A900D4A2A900D422A900D442A900B9
:100BC000C502A800C522A8006DFE07005723280013
:100BD0000E20ED00FEFF3A000000000068FE070056
:100BE000572328000E20ED00FEFF3A000000000011
:100BF00063FE0700572328000E20ED00FEFF3A0099
:100C000000000000D422A900D442A900C502A80017
:100C1000C522A9005AFE0700572328000E20ED0028
:100C2000FEFF3A0000000000D422A900D442A9002F
:100C3000C502A800C522A90051FE070057232800BD
:100C40000E20ED00FEFF3A0000000000D422A800B4
:100C5000D442A900C502A900C522A90048FE070088
:100C6000572328000E20ED00FEFF3A000000000090
:100C70008AC0B300F6FD07001AC0B300F4FD0700F8
:100C8000CAC0B300F2FD07002AC0B300F0FD0700A0
:100C9000EAC0B300EEFD0700FAC0B300ECFD0700A8
:080CA0004F057800000006007A
:10058000070120000E20ED00FEFF3A0000000000F1
:1005900000000000D462A800070120000E20ED003A
:1005A000FEFF3A000000000000000000D462A90035
:1005B000070120000E20ED00FEFF3A0000000000C1
:0805C00000000000000006002D
:10045000EBFF0700D482A900D4A2A90014E0AE00EB
:10046000D422A90014E0AF00D422A80014C0AE002A
:10047000D442A90014C0AF00D442A80014A0AE001A
:10048000C502A90014A0AF00C502A8001480AE00E8
:10049000C522A9001480AF00C522A80038000700BB
:1004A0001460AE00D422A9001460AF00D422A800CA
:1004B0001440AE00D442A9001440AF00D442A800BA
:1004C0001420AE00C502A9001420AF00C502A80088
:1004D0001400AE00C522A9001400AF00C522A80078
:0804E0002700070000000600E0
:10040000C122A800C102A800D042A800D022A800A2
:10041000D482A800D4A2A900D462A80007012000B9
:100420000E20ED00FEFF3A0000000000000000007A
:10043000D222AE0001003700FDFF3700C122A90023
:10044000C102A900D042A900D022A90000000600E4
:100B2C008A1F78000AC4B30046FE07004F05780000
:100B3C000220EF0000C4B300000CE10008003100FB
:100B4C000180FB00000045008A1F780010457800EA
:100B5C0062FE07004F0578000260EC00F5FF3700DD
:100B6C008A1F78000AC8B30036FE07004F057800CC
:040B7C00000006006F
:1004E800C5FF0700D4A2A800D482A90014E0AE007A
:1004F800D422A90014E0AF00D422A80014C0AE0092
:10050800D442A90014C0AF00D442A80014A0AE0081
:10051800C502A90014A0AF00C502A8001480AE004F
:10052800C522A9001480AF00C522A8001200070048
:100538001460AE00D422A9001460AF00D422A80031
:100548001440AE00D442A9001440AF00D442A80021
:100558001420AE00C502A9001420AF00C502A800EF
:100568001400AE00C522A9001400AF00C522A800DF
:0805780001000700000006006D
:100EB4000000FA00C035200080408800000E2000A9
:100EC40020A3B700CA50DD00003220001088700053
:100ED40001002E002032200001886500F0F321007B
:100EE40024A3B7003223EF003023EF0021E3A8004E
:080EF4000080FA000000060076
:100DAC000220EF000180FB0000004500104078009D
:100DBC006004E100390032000180FB0000004500B6
:100DCC009041780061C140009040780010CEB30093
:100DDC00000CE10002003A0010C0B30029003700FB
:100DEC0090CEB300001CE10002003A0020C0B3001A
:100DFC002400370050CFB300001CE10002003A0081
:100E0C0030C0B3001F003700A0CFB300001CE100BE
:100E1C0002003A0040C0B3001A003700B0CFB30054
:100E2C00001CE10002003A0050C0B300150037006E
:100E3C0030CFB300001CE10002003A0060C0B300E8
:100E4C0010003700D0CEB300001CE10002003A00C5
:100E5C0070C0B3000B00370060CFB300001CE10082
:100E6C0002003A00F0CEB30006003700C0CFB3004A
:100E7C00001CE10002003A0050CFB3000100370023
:100E8C00034078008A1F78000045780093FD070026
:100E9C004F05780082407800C2FF37001080200098
:080EAC00014878000000060077
:100D44008A1F7800D482A900D4A2A9000C0037001D
:100D54000AC8B300BDFD0700110037000ACCB30078
:100D6400BAFD07000E0037000AC9B300B7FD07003B
:100D74000B0037000ACDB300B4FD070008003700AC
:100D84006154E100F2FF32006254E100F3FF3200EB
:100D94006354E100F4FF32006454E100F5FF3200D3
:080DA4004F0578000000060075
:1005F0008A1F78007054E1000100390004003700C0
:100600000A80FB007000100000457800EEFF070034
:080610004F0578000000060010
:1005C8006054E100070036008A1F78000AC2B300B1
:1005D800C3FF07004F0578006140550000457800CB
:0805E800F7FF370000000600D8
:100618000200FA00823E2000110009000205D800FD
:100628008000780020802000014878008180FB004D
:10063800803E20000088B90000005500000798009F
:100648000005780042062000110009000200D800C9
:1006580080007800D0802000014878008180FB006D
:10066800400620000089B9000E00900002005000EA
:100678000007980000057800A2002000110009007A
:100688000200D800800078008080200001487800AF
:10069800A20020000E009000110009000200D800FE
:1006A800E0802000014878000080FA000000060081
:100718008A1F7800208020001004E00007003200C3
:10072800208020009080FB00000320000080400013
:10073800004578006AFF0700020037000AC2B300CC
:1007480067FF0700208020001004E00006003A0040
:10075800D08020001004E00003003A000AC2B30071
:100768005FFF070006003700D08020009080FB0064
:1007780000032000008040000045780058FF070073
:10078800208020001004E00009003A00D0802000FA
:100798001004E00006003A00808020001004E00009
:1007A80003003A000AC2B3004DFF070006003700F5
:1007B800808020009080FB00000320000080400023
:1007C8000045780046FF0700E08020009080FB008D
:1007D80000032000008040000045780040FF07002B
:1007E8001180200040C0B300804878004F05780091
:0407F80000000600F7
:1006B8000000FA00100020000A00DD008080EA0037
:1006C800C0322000108860004A1988002023A80042
:1006D8002003AF0001003700FDFF37002003A90009
:0C06E8000083BF000080FA000000060044
:101508000A8020000B002000090009000B1D78004C
:0415180000000600C9
:10151C00018020001015280002000900B058780046
:10152C00418020004015280000000900B018780008
:10153C003180200060152800B058780061802000B0
:10154C00E011280004000900B01878000000060023
:1014D0003400F8003600F800801F7800200020005B
:1014E0000C000900B01F780082FC0700A00120005A
:1014F0000C0009004F1078004F0078003600F9000A
:081500003400F9000040060070
:1006F4008680A900CAA2AE00030037000080200053
:100704001004A00002003700008020001014A00094
:0407140000000600DB
:101498003400F8003600F800801F78002000200093
:1014A8000C000900B01F7800D2FC0700A001200042
:1014B8000C0009004F1078004F0078003600F90042
:0814C8003400F90000400600A9
:1007FC0071FF2F004008200010886000C08020008E
:10080C00104078006404E10022003900C18020000F
:10081C000020EF0080487800F080200090407800A5
:10082C000060EF000220AF000060EC000080FB00D5
:10083C004101DD00F0802000904078000060EF0066
:10084C000200AF000060EC000080FB0002014000E1
:10085C00F0802000904078000060EF000240AF0074
:10086C000060EC000080FB004200DD000001410054
:10087C00F0802000904078000060EF000260AF0034
:10088C000060EC000080FB00C300DD002081200034
:10089C000148410047003700D2E2AF0003003700A7
:1008AC00308020001004A0000200370030802000AF
:1008BC001004A100D2C2AF0003003700F08020006A
:1008CC001004A00002003700F08020001004A100EA
:1008DC00D502A800D522A90047003700D2E2AF000C
:1008EC0003003700308020001014A00002003700F5
:1008FC00308020001014A100D2C2AF0003003700DA
:10090C00F08020001014A00002003700F0802000BE
:10091C001014A100D502A900D522A800360037007A
:10092C00D2E2AF0003003700308020001024A0007A
:10093C0002003700308020001024A100D2C2AF008A
:10094C0003003700F08020001024A00002003700C4
:10095C00F08020001024A100D502A800D522A80008
:10096C0025003700D2E2AF000300370030802000B2
:10097C001034A00002003700308020001034A10099
:10098C00D2C2AF0003003700F08020001034A0006A
:10099C0002003700F08020001034A100D502A9001D
:1009AC00D522A90014003700D502A900D522A90030
:1009BC0011003700C0802000104078006004E10076
:1009CC00B5FF3200C0802000104078006104E100C7
:1009DC00C2FF3200C0802000104078006204E100A9
:1009EC00CFFF3200C0802000104078006304E1008B
:1009FC00DCFF3200ECFF370011C0B300C0802000D8
:100A0C0010C8400011002000A08020001088400079
:100A1C0051408000401F20000008E10003003A0014
:100A2C000020EF0050408800CDC2AA001100200029
:100A3C0060802000108840003140800000F42100CC
:100A4C000008E10002003A000020EF00304088006E
:100A5C003140800000FA20000008E1000300310062
:100A6C00008020001034A10002003700008020001C
:100A7C001034A00011C0B3009080200010C84000BA
:100A8C0090802000104078006204E10023003A00BE
:100A9C0000802000104078000020AE0008003700D5
:100AAC00008020001014A100204080006000E100B4
:100ABC000300360011002000408020001088100038
:100ACC0000802000104078000000AE0009003700C4
:100ADC00008020001004A10041062000408020006E
:100AEC001008E100030036001100200040802000B7
:100AFC0010884000918020000020EF008048780092
:100B0C00CA62AF0003003700008020001024A00050
:100B1C0002003700008020001024A1000000060015
:020000040001F9
:1000080000000000000000000000000000000000E8
:10001800020400000E0100000F1100000F00000094
:10002800020400000E1100001F1000000E00000066
:10003800050A0000000E0000111100000E0000006B
:100048000204000011110000111300000D0000004F
:10005800050A000011110000111300000D00000036
:10006800020400000E110000111100000E00000033
:10007800020400000C040000040400000E0000004C
:10008800352E00002052000047420000204C00009E
:100098004544000020740000657300007A74000075
:1000A800003400002E200000506F0000746500002E
:1000B8006E630000696F00006DE900007465000060
:0400C80072000000C2
:1000CC0053E1000072670000612000004C45000005
:1000DC0044200000766900006C6C00006F67000023
:1000EC00003100002E2000004C450000442600008A
:1000FC004C4300004420000074650000737A00003B
:04010C00740000007B
:10011000473100003D50000020470000323D000004
:100120005A200000473300003D5000005A000000F4
:10013000332E0000204600006F72000067F30000BD
:10014000206A0000656C000061640000F30000009C
:100150004D6900006E640000656E000020720000B2
:10016000656E000064620000656E00003F000000E4
:1001700048610000206500007A740000206F0000D4
:100180006C760000617300006F6400000050000096
:10019000494300002032000034200000702E00008F
:0C01A000706100006E6500006C00000043
:1001AC00322E0000204700006F6D0000622000001E
:0C01BC0074650000737A000074000000FD
:1001C800454E0000435F0000473D0000746F00008B
:1001D80076E1000062620000006A0000F32000007F
:1001E800612000006B6900006A6500006C7A0000FD
:0401F800F50000000E
:1001FC0054650000737A00007420000076E900005A
:10020C0067650000004500005F4700003D7400007A
:0C021C006F760000E1620000620000004C
:10022800473400003D7400006F760000E162000072
:040238006200000060
:04023C0000000000BE
:0402400000000000BA
:0402440000000000B6
:0402480000000000B2
:04024C0000000000AE
:1002500050490000524F0000533D0000426500002D
:100260000047000052450000454E00003D4200009E
:040270006500000025
:100274005AF600004C4400003D42000065000000B6
:10028400424C0000554500003D420000650000005E
:1002940052450000443D000042650000000000009B
:0402A4000000000056
:0402A8000000000052
:0402AC00000000004E
:0200000401F009
:20000000CF000000CF0000000700000082000000A50000005F000000F7000000C3000000FB
:00000001FF
